:0600000000008A013C280B
:0800080009005434653473341F
:100010007434203452346F3476346534723420347E
:10002000763431342E343134003428346334293476
:10003000323430343034343420344534723469341A
:10004000633420344C3475346E3464347134753414
:1000500069347334743400347734653469347234F9
:1000600064342034623475346D3470342034763422
:1000700061346C343A3400348330831603138100C6
:1000800083128B120B17313090006030F8009822E9
:1000900049280530F0000030F100AE220D30A222D8
:1000A0000A30A2221530F0000030F100AE220D30EF
:1000B000A2220A30A22283120313FA148316861096
:1000C00083127A158316061183127A168316061286
:1000D0008312031306168316061283127A167A10F9
:1000E000831606148312FA118316861583120030C4
:1000F000A0000030A1000030A2000030A3000108E1
:10010000F000F1017008AC007108AD007008B92270
:100110007108B922861D91280130F0000030F100ED
:100120009328F001F1010130F2000030F300C22207
:100130007008F2007108F300CB22F100CB22F0002E
:1001400083120313061CA9280130F0000030F100CF
:10015000AB28F001F101D222831203137008A4002E
:100160007108A5002408F0002508F1000030700691
:100170000319E028013070060319DA2802307006EE
:100180000319DD28033070060319D7282C30F0003E
:100190000030F100AE22831203132408F00025087A
:1001A000F100DB220D30A2220A30A2220F291221F7
:1001B00049210F297E2149210F299E2112210F2932
:1001C0009E217E21BE21831203132C08F0002D08EE
:1001D000F1001723831203137008AC007108AD00FF
:1001E0002C08F0002D08F1000330F2000030F3007D
:1001F0003423831203137008A4007108A500240897
:10020000F0002508F100003070060319DA280130EB
:1002100070060319DD28023070060319E028BE219C
:1002200086280000831203132008F0002108F10043
:100230000130F2000030F300D22283120313700861
:10024000A0007108A1002008F0002108F100003092
:10025000F2008030F3009C23F201F30183230319A1
:1002600032290800831203132008F0002108F1004E
:100270000A30F2000030F3009C23F201F3018323E3
:1002800003194829831203130A30A0000030A1008B
:1002900008002208F0002308F1000130F2000030CD
:1002A000F300D222831203137008A2007108A30086
:1002B0002208F0002308F1000030F2008030F30043
:1002C0009C23F201F3018323031967290800831299
:1002D00003132208F0002308F1000A30F200003076
:1002E000F3009C23F201F301832303197D29831278
:1002F00003130A30A2000030A30008002008F00019
:100300002108F1000130F2000030F3002D238312A8
:1003100003137008A0007108A1000A30F200003039
:10032000F3009C23F201F301832303199D29831217
:100330000313F630A000FF30A10008002208F000EF
:100340002308F1000130F2000030F3002D23831266
:1003500003137008A2007108A3000A30F2000030F5
:10036000F3009C23F201F30183230319BD298312B7
:100370000313F630A200FF30A30008000030F000A5
:100380000030F1002208F2002308F3002D2383122D
:1003900003137008A6007108A7002608F0002708BC
:1003A000F1000030F2008030F3009C23F201F301F1
:1003B00083230319032A7008B9227108B922003077
:1003C000F0000030F100831203132608F200270822
:1003D000F3002D231930F2000030F300F7227008EB
:1003E000F2007108F300CB22F100CB22F000EE30D6
:1003F000F0000230F1002D23831203137008A800CF
:100400007108A900232A7008B9227108B9222608A8
:10041000F0002708F1001930F2000030F300F72255
:100420007008F2007108F300CB22F100CB22F0003B
:10043000EE30F0000230F100D22283120313700874
:10044000A8007108A9000130F4000030F500280868
:10045000F0002908F100DE231430F0000030F10034
:100460000224831203132008F0002108F100003059
:10047000F2008030F3009C23F201F301832303197F
:10048000692A7008B9227108B9220030F0000030E2
:10049000F100831203132008F2002108F3002D233A
:1004A0001930F2000030F300F7227008F2007108F2
:1004B000F300CB22F100CB22F000EE30F00002304E
:1004C000F1002D23831203137008AA007108AB00FA
:1004D000892A7008B9227108B9222008F000210881
:1004E000F1001930F2000030F300F7227008F2003A
:1004F0007108F300CB22F100CB22F000EE30F000C7
:100500000230F100D222831203137008AA0071088E
:10051000AB000230F4000030F5002A08F0002B0890
:10052000F100DE231430F0000030F1000224080056
:10053000673083160313990018159816831218163E
:1005400098170800831203130C1EA42A99000800B0
:10055000700FF103F10AF00071040800B5220038B1
:1005600003190800A222A822AE2A71088A00700886
:1005700082008B13F9007808840079088000F80A5B
:100580008B1708000310F20803190800F00DF10D95
:10059000F20BC22A08008B13F803780884000008C5
:1005A0008B1708007208F00773080318730AF10725
:1005B00008002430A2227108D000500EE822500812
:1005C000E8227008D000500EE8225008E822080007
:1005D0000F39F63E0318073E0A3E303EA2220800BD
:1005E0007008F60771080318710AF7070800F6018A
:1005F000F701F401F50170087104031D002B0034AC
:10060000720873040319122B721C0B2BF022031CAB
:100610000B2BF40DF50D0310F30CF20C0310F00D81
:10062000F10D002B7608F0007708F10000340D3052
:10063000F200F301F722EB30F2000C30F300D2228B
:1006400008000310F20DF30DF40B212B080003102A
:10065000F30CF20CF40B272B08007208F00273085D
:10066000031C730AF1020800F601F7017208730413
:100670000319FF340130F40073080038031D4B2BBD
:100680007208013A031D4B2B7008F6007108F70041
:10069000F001F101003470087104031D502B003487
:1006A000F31B5B2BF40A7408B9220130F4002123F8
:1006B000CB22F400502B7208B9227308B9227608B5
:1006C000F2007708F3007408B9220130F400212306
:1006D000CB22F4007208F6007308F700CB22F30077
:1006E000CB22F2002D230318772BD222782B7614FD
:1006F000F403031900347408B9220130F4002723ED
:10070000CB22F4005B2B73087102031D08007208F2
:10071000700208008323031C902BF001F1010800F4
:100720000130F000F10108008323031D8A2B902B78
:100730008323031D9C2B902B832303198D2B0318DC
:10074000902B8D2B832303198D2B902BF001F1011E
:100750008323031D902B8D2B7008F2007108F3008A
:100760000130F000F101C2220800AC23831603130C
:100770007008860471088704FF30F006F1067008DF
:100780008312860571088705700883168605700830
:1007900087050800AC23831203137008FA0471085C
:1007A000FB047008860471088704FF30F006F10628
:1007B0007008831686057108870508007008F20026
:1007C0007108F300FF30F000F1002D237008831250
:1007D00003138E0071088F007408F000F101CA2322
:1007E000831203130C100C1CF32B0C107408F00074
:1007F000F101B5230800F003700FF10AF10370084E
:1008000071040800831203130B110B1D052CFB232D
:06081000031D022C08008C
:00000001FF
